:1000000000308A00E72C0000FF00030E8301A100EE
:100010000A08A0008A010408A2007708A300780853
:10002000A4007908A5007A08A6007B08A70083131E
:1000300083128C308400001D1F280C1932282208DE
:1000400084002308F7002408F8002508F900260892
:10005000FA002708FB0020088A00210E8300FF0E0B
:100060007F0E09008A110A1235281430AB0083165E
:100070000814831208183F285030AE004928831610
:1000800008158312081947285F30AE00492801304F
:10009000AE00831688158312881951285030AF009E
:1000A0005B28831688148312881859285F30AF00A4
:1000B0005B280130AF000808F038B000FF30B10015
:1000C000831608168312081A6628B0138316881739
:1000D0008312881B6C2830128316061483120618AC
:1000E0007228311383168614831286187828B11269
:1000F00083160615831206197E28B11383168615FA
:100100008312861984283112831606168312061A62
:100110008A283111831686168312861A9028311088
:10012000831606178312061B9628B11083168617AE
:100130008312861B9C28B1110C118A110A121F28E8
:100140003F3085008601FF3087008801890120301B
:1001500083168500FF3086001F3087008312DE0083
:10016000FF3083168800091089100911811383124A
:100170001F0838399F00063083169F00831294129F
:10018000DE125E088316870083125E165E088316F1
:10019000870085168312DE155E08831687003430CB
:1001A0008312940000308316940083120711970184
:1001B0000530970083160C15C03083128B04A801FC
:1001C000A901AA011430AB000130AE000130AF002C
:1001D0008A110A12F12C0830F700F70BED2883166C
:1001E0000512831205120330F700F70BF52883166A
:1001F0000516831200345E155E088316870083128D
:100200000719FB28AB012B08033C031C5429831658
:1002100014180C298312072983121308AC009413B5
:1002200014132B08F700F70803192329013077026C
:1002300003192C290230770203192F290330770282
:100240000319332942294230AD002C08803C0319A0
:100250002B291430AB0045295A30AD004529080838
:100260006038AD0045290608AD003308C23C031DC7
:1002700041292C08803C031D41290230A80014307C
:10028000AB004529FF30AD0045292D0893003230E1
:100290002B0784002C08800048302B0784002D0891
:1002A0008000EB20AB0A03298A110A12042D5E1587
:1002B0005E0883168700831207195729AB012B08A4
:1002C000073C031CC7298316141868298312632965
:1002D00083121308AC00941314132B08F700F708CB
:1002E00003198F2901307702031998290230770208
:1002F00003199B290330770203199E2904307702E2
:100300000319A129053077020319A42906307702C1
:100310000319A729073077020319AA29B529CE3076
:10032000AD002C08803C031997291430AB00B82984
:100330005A30AD00B8293008AD00B8293108AD00F9
:10034000B8290130AD00B8290130AD00B8292E0818
:10035000AD00B8292F08AD003308C23C031DB429F5
:100360000230A8001430AB00B829FF30AD00B82926
:100370002D08930032302B0784002C088000483071
:100380002B0784002D088000EB20AB0A5F298A111F
:100390000A12062D02302B02FA3E0318E729063E08
:1003A000EA29C030AD00E7294030AD00E729A908AF
:1003B000031DDC29AD01DE298030AD00E729403086
:1003C000AD00E7298030AD00E729AD01E7298A11AA
:1003D0000A12FD2B0A148A100A118207D129D42986
:1003E000D729DF29E229E52902302B02FA3E03183A
:1003F0001C2A063E1F2AAD011C2AAD011C2A803092
:10040000AD001C2AB508031D082A4030AD000A2A99
:100410008030AD001C2AB508031D102AAD01122A38
:100420008030AD001C2AB508031D192A5030AD00DC
:100430001B2A2830AD001C2A8A110A12FF2B0A1031
:100440008A140A118207FB29FD29FF29022A0B2A97
:10045000132A02302B02FA3E03183E2A063E412A96
:10046000AD013E2AAD013E2A4030AD003E2AAD012D
:100470003E2A8030AD003E2AAD013E2A8A110A1282
:10048000012C0A108A140A118207302A322A342ACF
:10049000372A392A3C2A02302B02FA3E0318652AF1
:1004A000063E682AAD01652AAD01652AAD01652ABF
:1004B000B508031D5E2A2030AD00602AE030AD0093
:1004C000652AAD01652AAD01652A8A110A12032C3D
:1004D0000A108A140A118207522A542A562A582AC4
:1004E000612A632A02302B02FA3E0318962A063E3E
:1004F000A42AAA08031D7F2AFF30AD00802AAD017F
:10050000962AAA08031D872AFF30AD00892A803069
:10051000AD00962AFF30AD00962AFF30AD00962A36
:10052000FF30AD00962AFF30AD00962AB508031DB6
:10053000A02A3608803C031DA02A0130AA00A12A67
:10054000AA018A110A12052C0A108A140A118207BC
:10055000792A812A8A2A8D2A902A932AA908031D9A
:10056000C52A02302B02FA3E0318C42A063EE62AA8
:10057000AD01C42AAD01C42AAD01C42AAD01C42A0B
:10058000AD01C42AAD01C42AE32A290BC82ACC2A0A
:100590002908023C031DE32A02302B02FA3E03180D
:1005A000E32A063EF02AFF30AD00E32AFF30AD001B
:1005B000E32AC030AD00E32AAD01E32AAD01E32A0E
:1005C0005A30AD00E32A8A110A12072C0A108A1445
:1005D0000A118207B82ABA2ABC2ABE2AC02AC22A0D
:1005E0000A108A140A118207D32AD62AD92ADC2AA9
:1005F000DE2AE02A02302B02FA3E03180D2B063EBB
:10060000212BAD010D2BAD010D2BAD010D2BAD013E
:100610000D2BAD010D2BAD010D2BB508031D1E2BB0
:100620002908FD3E03181E2B033E2B2BA8011E2B71
:100630000130A8001E2B0330A8001E2B8A110A12BD
:10064000092C0A148A140A118207012B032B052B8B
:10065000072B092B0B2B0A148A140A118207162B5D
:10066000182B1B2B02302B02FA3E0318452B063E9B
:10067000532BAD01452BAD01452BAD01452BAD01F4
:10068000452BAD01452BAD01452B3508803C031DA5
:100690004C2B0130A900502BB508031D502BA9018C
:1006A0008A110A120B2C0A148A140A118207392B98
:1006B0003B2B3D2B3F2B412B432B02302B02FA3E91
:1006C0000318712B063E762BAD01712BAD01712BFA
:1006D000AD01712BAD01712BAD01712B5A30AD0005
:1006E000712B0230A9008A110A120D2C0A148A14E7
:1006F0000A118207642B662B682B6A2B6C2B6E2BDE
:1007000002302B02FA3E0318952B063E982BAD01C2
:10071000952BAD01952B4030AD00952BAD01952B60
:10072000AD01952B5A30AD00952B8A110A120F2C72
:100730000A148A140A118207872B892B8B2B8E2B84
:10074000902B922B5E155E08831687008312071983
:10075000A22BAB012B08073C031C252C8316141875
:10076000B32B8312AE2B83121308AC009413141313
:10077000AB08031DC42BCF30AD002C08803C0319FF
:10078000C32B1430AB00162C2B0BC92B5A30AD00E9
:10079000162C2B08013C0318142C2B08073C031CB7
:1007A000142C3308F700A23077020319FC2B6230B7
:1007B00077020319FE2BE23077020319002C323046
:1007C00077020319022CB23077020319042C82300D
:1007D00077020319062CC23077020319082C223045
:1007E000770203190A2CF230770203190C2C02301D
:1007F000770203190E2C102CCA29132CF429132C60
:10080000292A132C4B2A132C722A132CAE2A132CB0
:10081000FA2A132C322B132C5D2B132C802B132C28
:10082000FF30AD00132C162C1430AB002D089300B4
:1008300032302B0784002C08800048302B078400BE
:100840002D088000EB20AB0AAA2B8A110A12082D72
:100850005E155E088316870083120719282CAB01EA
:100860002B08133C031CE42C83161418392C831218
:10087000342C83121308AC00941314132B08F700C4
:10088000F7080319902C013077020319992C0230D4
:10089000770203199C2C033077020319A02C043033
:1008A00077020319A22C053077020319A52C063014
:1008B00077020319A82C073077020319AB2C0830F4
:1008C00077020319AE2C093077020319B02C0A30D5
:1008D00077020319B22C0B3077020319B42C0C30B9
:1008E00077020319B62C0D3077020319B82C0E309D
:1008F00077020319BA2C0F3077020319BC2C103081
:1009000077020319BE2C113077020319C02C123064
:1009100077020319C22C133077020319C42CD22C8E
:100920009E30AD002C08803C0319982C1430AB008D
:10093000D52C5A30AD00D52C08086038AD00D52C28
:100940000608AD000130AD00D52C0130AD00D52C2E
:100950000130AD00D52C0130AD00D52CAD01D52C2A
:10096000AD01D52CAD01D52CAD01D52CAD01D52CCB
:10097000AD01D52CAD01D52CAD01D52CAD01D52CBB
:10098000AD01D52CAD01D52CAD013308C23C031D02
:10099000D12C3508803C031DD12C0230A800143026
:1009A000AB00D52CFF30AD00D52C2D089300323094
:1009B0002B0784002C08800048302B0784002D086A
:1009C0008000EB20AB0A302C8A110A120A2D840118
:1009D0001F308305073083169F00FF308312DE002F
:1009E000A0282808F700F7080319032D0130770223
:1009F0000319052D023077020319072D0330770202
:100A00000319092D0B2DFB280C2D57290C2DA22B7A
:0C0A10000C2D282C0C2D0C2DF12C63005B
:02400E00723FFF
:00000001FF
